:08369F0033302E3320202000FF
:10315600C107C10842035D000444032600000000C5
:1031660044032A0000000044032E0000000044032C
:1031760032000000004403360000000044033A0019
:1031860000000044033E000000004403420000002B
:0631960000420346000A9E
:1035E100758850758922758E0C758AAE758CAE758D
:0635F1008BC7758DC72297
:1035F70075F1FEE4F5F2F5F375A41A75D41175E1CA
:053607000675E2C0227F
:10361D0075D10275BCA075E8C075BA1F43E60822C6
:0C36540075A14075F80175A202D2AE22EB
:0436CE0075B283222C
:0B36600075CA8275CBFDD2CAD2AD2224
:0D362D007592077593F875910443E68022AD
:10359A00E4F5D91236CE1235F712361D1236541208
:0835AA0035E112366002362DF6
:0B366B00E5B030E403C20122D20122CE
:081A2400E4FFE5B030E3010F1F
:011A2C002297
:10342A00EF25E0FFA201E4334F14601314600A147D
:10343A00600A240370097F36227F37227F35227F74
:02344A0034222A
:101A3000E4FDFF122A547D017F01122A547D027FAA
:101A400002122A547D037F03122A547D0A7F041256
:101A50002A547D0B7F05122A547D0C7F06122A54CE
:101A60007D0D7F07122A547D0E7F08122A547D0FA8
:101A70007F09122A54D3E5139430E5129403400BE6
:101A800090034FE4F0A37410F08046D3E513946400
:101A9000E5129402400B90034FE4F0A37408F08029
:101AA00030D3E5139498E5129401400B90034FE472
:101AB000F0A37404F0801AD3E51394CCE5129400DB
:101AC00090034FE44007F0A37402F08004F0A304F5
:101AD000F0D3E50F9430E50E9403400B900351E4EE
:101AE000F0A37410F08046D3E50F9464E50E9402E1
:101AF000400B900351E4F0A37408F08030D3E50F5D
:101B00009498E50E9401400B900351E4F0A3740403
:101B1000F0801AD3E50F94CCE50E9400900351E4C5
:101B20004007F0A37402F08004F0A304F0D3E50BA7
:101B30009430E50A9403400B900355E4F0A374D06D
:101B4000F08047D3E50B9464E50A9402400B9003C0
:101B500055E4F0A374C8F08031D3E50B9498E50AFE
:101B60009401400B900355E4F0A374C4F0801BD3A0
:101B7000E50B94CCE50A9400900355E44007F0A3EC
:101B800074C2F08005F0A374C1F0D3E51B9430E576
:101B90001A9403400B900353E4F0A374D0F08047F1
:101BA000D3E51B9464E51A9402400B900353E4F0D0
:101BB000A374C8F08031D3E51B9498E51A940140D2
:101BC0000B900353E4F0A374C4F0801BD3E51B9483
:101BD000CCE51A9400900353E44007F0A374C2F0DC
:101BE0008005F0A374C1F0E5097003021C96D3E5EB
:101BF000179430E5169403400890035B7410F0804E
:101C00003CD3E5179464E5169402400890035B7496
:101C100008F08029D3E5179498E5169401400890C0
:101C2000035B7404F08016D3E51794CCE51694009A
:101C300090035B40057402F080037401F0D3E5115A
:101C40009414E5109403400890035BE044A0803BAB
:101C5000D3E5119454E5109402400890035BE044EE
:101C6000808028D3E51194A4E510940140089003E6
:101C70005BE044608015D3E51194ECE5109400908E
:101C8000035BE04004444080024420FF900359E499
:101C9000F0A3EFF08007E4900359F0A3F0E508709B
:101CA00003021D4BD3E51D9430E51C9403400890BE
:101CB000035B7410F0803CD3E51D9464E51C940232
:101CC000400890035B7408F08029D3E51D9498E5E3
:101CD0001C9401400890035B7404F08016D3E51D4A
:101CE00094CCE51C940090035B40057402F08003E3
:101CF0007401F0D3E5199414E51894034008900397
:101D00005BE044A0803BD3E5199454E5189402406D
:101D10000890035BE044808028D3E51994A4E5187B
:101D20009401400890035BE044608015D3E519946A
:101D3000ECE518940090035BE040044440800244CA
:101D400020FF900357E4F0A3EFF022E4900357F054
:031D5000A3F022DB
:101D530012359A121A247523079002E67407F0A32A
:101D630074D0F012366B12342A900348EFF0123617
:101D73004743F60130010543A480C287D2AF123531
:101D8300801233913002051208A7C202E52660399A
:101D930014601414600924FE702C6309018003632A
:101DA300080112352E801F30070F300105A287B3BB
:101DB3009287308711C20C800DE4900361F01236D4
:101DC300C3300102C287E4F526300810900348E0CF
:101DD300FF7BFF7A36799F1231B6C2087B017A0204
:101DE3007964123365EF609C900266E01218CF1E8F
:101DF30067041EAE051E29141E11161E1E171E2E65
:101E03001A1E501B1E5B1D1E611E00001EFE2001BC
:101E130003021EFED287C20C021EFE200103021E15
:101E2300FEC287021EFED207021EFE7B017A0279E2
:101E330064900274EBF0A3EAF0A3E9F0121670FECB
:101E4300900348E0FF6E6003021EFE800590034886
:101E5300E0FF12348F021EFE1236B6021EFE123649
:101E6300BD021EFE7B017A027964900277EBF0A338
:101E7300EAF0A3E9F0900003121689FF900348E00B
:101E83006F707830876D90027704F0A3EAF0A3E9CE
:101E9300F0900005121689FF900006121689FD9036
:101EA3000004121689FB122E4A80487B017A0279BC
:101EB30064900277EBF0A3EAF0A3E9F09000031239
:101EC3001689FF900348E06F7031308726900277C0
:101ED30004F0A3EAF0A3E9F0900005121689FF903D
:101EE3000006121689FD900004121689FB121921AF
:101EF300123391900348E0FF1234F1208703021D4F
:101F0300DF900266E014603424FA60531470030215
:101F13001FB024066003021DDF12360C7B017A0218
:101F23007964900274EBF0A3EAF0A3E9F090000364
:101F3300121689900361F01236C3806B12360C7B44
:101F4300017A027964900274EBF0A3EAF0A3E9F05A
:101F5300900003121689900361F0123391804812A6
:101F6300360C7B017A02796490027AEBF0A3EAF0F3
:101F7300A3E9F0900003121689FF9000041216895A
:101F8300FD900005121689FBC00390027AE0FBA3C3
:101F9300E0FAA3E0F9900006121689900280F0D0CF
:101FA30003122D9612339112368B021DDF12360C5B
:101FB3007B017A02796490027AEBF0A3EAF0A3E959
:101FC300F0900003121689FF900004121689FD9009
:101FD3000005121689FB1223D612339112368B0297
:021FE3001DDF00
:102FEE00E5B05407F5226523600CE5226523F52430
:102FFE00752503852223E52560361525E5257030D8
:10300E00E52430E211E52220E20C9003247405F051
:10301E00A374DCF0D200E52430E108E52220E103C0
:10302E00752602E52430E008E52220E0037526012E
:10303E00300027900325E024FFF0900324E034FFB6
:10304E00F0E5B054046005752604C200900324E038
:0A305E007002A3E07004C200D20863
:013068002245
:031A12000236C9D0
:0536C900C2CFD2023265
:1008A700E490035FF0900349A3E0F5A390035FE0B2
:1008B700C36480948540F590035DE4F0A37404F06D
:1008C700F5BB90033AE0FCA3E0FDA3E0FEA3E0FF45
:1008D700900326E0F8A3E0F9A3E0FAA3E02FFFEAEC
:1008E7003EFEE93DFDE83CFC90027D12189275E85A
:1008F700D03004FD30031DC2039002E6E07002A36E
:10090700E0600E9002E7E024FFF09002E6E034FF9B
:10091700F0121A309002D1E0250DFF9002D0E03599
:100927000CFEE4FCFD90027D1218929002D7E025A0
:1009370015FF9002D6E03514FEE4FCFD900281120B
:100947001892E47FFF7E03FDFC90027DE0F8A3E0B0
:10095700F9A3E0FAA3E0FBD312185B400A90027DEB
:1009670012189E000003FFE47FFF7E03FDFC900248
:1009770081E0F8A3E0F9A3E0FAA3E0FBD312185B48
:10098700400A90028112189E000003FF90027DE04A
:10099700F8A3E0F9A3E0FAA3E0FBC374FF9BFB74A1
:1009A700039AFAE499F9E498F89002CEE0FEA3E0FE
:1009B700FFE4FCFD121728780A12186CC004C00562
:1009C700C006C0079002D2E0FEA3E0FFE4FCFD9062
:1009D700027DE0F8A3E0F9A3E0FAA3E0FB121728F1
:1009E700780A12186CD003D002D001D000EF2BFF89
:1009F700EE3AFEED39FDEC38FC9002851218929024
:100A07000281E0F8A3E0F9A3E0FAA3E0FBC374FFD7
:100A17009BFB74039AFAE499F9E498F89002D4E0FE
:100A2700FEA3E0FFE4FCFD121728780A12186CC039
:100A370004C005C006C0079002D8E0FEA3E0FFE4AB
:100A4700FCFD900281E0F8A3E0F9A3E0FAA3E0FB44
:100A5700121728780A12186CD003D002D001D000E0
:100A6700EF2BFFEE3AFEED39FDEC38FC90028912D0
:100A7700189290032AE0FCA3E0FDA3E0FEA3E0FFA9
:100A8700900285E0F8A3E0F9A3E0FAA3E0FBD31214
:100A9700185B4035900285E0FCA3E0FDA3E0FEA3D0
:100AA700E0FF90032A121892900285E0FCA3E0FD74
:100AB700A3E0FEA3E024FCFFEE34FFFEED34FFFDD0
:100AC700EC34FFFC9003328052900332E0FCA3E049
:100AD700FDA3E0FEA3E0FF900285E0F8A3E0F9A301
:100AE700E0FAA3E0FBC312185B5033900285E0FCE9
:100AF700A3E0FDA3E0FEA3E0FF900332121892905B
:100B07000285E0FCA3E0FDA3E0FEA3E02404FFE4EC
:100B17003EFEE43DFDE43CFC90032A12189290034C
:100B27003AE0FCA3E0FDA3E0FEA3E0FF900289E02A
:100B3700F8A3E0F9A3E0FAA3E0FBD312185B403572
:100B4700900289E0FCA3E0FDA3E0FEA3E0FF900391
:100B57003A121892900289E0FCA3E0FDA3E0FEA3FD
:100B6700E024FCFFEE34FFFEED34FFFDEC34FFFC28
:100B77009003428052900342E0FCA3E0FDA3E0FE15
:100B8700A3E0FF900289E0F8A3E0F9A3E0FAA3E06D
:100B9700FBC312185B5033900289E0FCA3E0FDA36E
:100BA700E0FEA3E0FF900342121892900289E0FC56
:100BB700A3E0FDA3E0FEA3E02404FFE43EFEE43D42
:100BC700FDE43CFC90033A121892900332E0FCA338
:100BD700E0FDA3E0FEA3E0FF9002851218929003C8
:100BE70042E0FCA3E0FDA3E0FEA3E0FF9002891230
:100BF7001892E47FFF7E03FDFC900285E0F8A3E0F6
:100C0700F9A3E0FAA3E0FBD312185B400A90028530
:100C170012189E000003FFE47FFF7E03FDFC900295
:100C270089E0F8A3E0F9A3E0FAA3E0FBD312185B8D
:100C3700400A90028912189E000003FFE50970031D
:100C4700020F549002CCE0FEA3E0FFE4FCFD90020B
:100C570085E0F8A3E0F9A3E0FAA3E0FBC312185B71
:100C67004003020D7C900285E0FCA3E0FDA3E0FEBB
:100C7700A3E0FF780A12187F90028D121892900253
:100C87008DE0FCA3E0FDA3E0FEA3E0FFC006C007E4
:100C9700AE10AF11AB07AA06E4F9F8D007D00612D9
:100CA70017B390028D12189290028DE0F8A3E0F925
:100CB700A3E0FAA3E0FBAE16AF17E4FCFD1217287A
:100CC70090028D12189290028DE0FCA3E0FDA3E044
:100CD700FEA3E0FF780A12186C90028D121892900A
:100CE7000285E0FCA3E0FDA3E0FEA3E0FF780A1283
:100CF700187F900299121892900299E0FCA3E0FDE8
:100D0700A3E0FEA3E0FFC006C007AE10AF11AB071C
:100D1700AA06E4F9F8D007D0061217B39002991281
:100D27001892E47FFF7E03FDFC900299E0F8A3E0B0
:100D3700F9A3E0FAA3E0FBC312185B9002995019DC
:100D4700E0F8C374FF9BFF74039AFEE499FDE498EF
:100D5700FC900299121892800712189E000000005A
:100D6700900299E0F8A3E0F9A3E0FAA3E0FBAE0E46
:100D7700AF0F020F11AE10AF11E4FCFD900285E03A
:100D8700F8A3E0F9A3E0FAA3E0FBD312185B402A2B
:100D9700AE10AF11AB07AA06900285E0FCA3E0FDF9
:100DA700A3E0FEA3E09BFFEE9AFEED9400FDEC941A
:100DB70000FC90028D121892800A90028D12189EE4
:100DC7000000000090028DE0FCA3E0FDA3E0FEA37D
:100DD700E0FF780A12187F90028D121892C3E5116E
:100DE70094FFE5109403503BC374FF9511FF740300
:100DF7009510FEE4FCFD90029912189290028DE086
:100E0700FCA3E0FDA3E0FEA3E0FF900299E0F8A3B6
:100E1700E0F9A3E0FAA3E0FB1217B390028D1218D2
:100E270092800A90029912189E0000000090028D8D
:100E3700E0F8A3E0F9A3E0FAA3E0FBAE0AAF0BE406
:100E4700FCFD12172890028D12189290028DE0FC7B
:100E5700A3E0FDA3E0FEA3E0FF780A12186C90025E
:100E67008D121892E47FFF7E03FDFC900285E0F867
:100E7700A3E0F9A3E0FAA3E0FBC312185B501C90B0
:100E87000285E0F8C374FF9BFF74039AFEE499FDA3
:100E9700E498FC900299121892800A90029912180D
:100EA7009E00000000900299E0FCA3E0FDA3E0FE95
:100EB700A3E0FF780A12187F900299121892C3E5EF
:100EC7001194FFE5109403502F900299E0FCA3E0E2
:100ED700FDA3E0FEA3E0FFC006C007C374FF9511A2
:100EE700FF74039510AB07FAE4F9F8D007D00612A0
:100EF70017B3900299121892900299E0F8A3E0F9BB
:100F0700A3E0FAA3E0FBAE16AF17E4FCFD12172827
:100F1700900299121892900299E0FCA3E0FDA3E0D9
:100F2700FEA3E0FF780A12186C90029912189290AB
:100F3700028DE0FCA3E0FDA3E0FEA3E0FF90029991
:100F4700E0F8A3E0F9A3E0FAA3E0FB80599002855B
:100F5700E0F8A3E0F9A3E0FAA3E0FBC374FF9BFB6F
:100F670074039AFAE499F9E498F8AE0EAF0FE4FC2B
:100F7700FD121728780A12186CC004C005C006C0F5
:100F870007AE0AAF0BE4FCFD900285E0F8A3E0F999
:100F9700A3E0FAA3E0FB121728780A12186CD00313
:100FA700D002D001D000EF2BFFEE3AFEED39FDEC79
:100FB70038FC90028D121892E50870030212C8AE31
:100FC70018AF19E4FCFD900289E0F8A3E0F9A3E06B
:100FD700FAA3E0FBC312185B40030210F4900289E6
:100FE700E0FCA3E0FDA3E0FEA3E0FF780A12187F70
:100FF700900291121892900291E0FCA3E0FDA3E009
:10100700FEA3E0FFC006C007AE18AF19AB07AA06DC
:10101700E4F9F8D007D0061217B39002911218928C
:10102700900291E0F8A3E0F9A3E0FAA3E0FBAE1C7D
:10103700AF1DE4FCFD12172890029112189290023E
:1010470091E0FCA3E0FDA3E0FEA3E0FF780A1218FD
:101057006C900291121892900289E0FCA3E0FDA324
:10106700E0FEA3E0FF780A12187F9002951218920B
:10107700900295E0FCA3E0FDA3E0FEA3E0FFC0061D
:10108700C007AE18AF19AB07AA06E4F9F8D007D026
:10109700061217B3900295121892E47FFF7E03FDA4
:1010A700FC900295E0F8A3E0F9A3E0FAA3E0FBC304
:1010B70012185B9002955019E0F8C374FF9BFF74F8
:1010C700039AFEE499FDE498FC9002951218928029
:1010D7000712189E00000000900295E0F8A3E0F9BF
:1010E700A3E0FAA3E0FBAE12AF13021287AE18AF6C
:1010F70019E4FCFD900289E0F8A3E0F9A3E0FAA364
:10110700E0FBD312185B402AAE18AF19AB07AA064B
:10111700900289E0FCA3E0FDA3E0FEA3E09BFFEEC5
:101127009AFEED9400FDEC9400FC90029112189247
:10113700800A90029112189E00000000900291E030
:10114700FCA3E0FDA3E0FEA3E0FF780A12187F905E
:101157000291121892C3E51994FFE51894035039C8
:10116700C374FF9519FF74039518FEE4FCFD900204
:1011770095121892900291E0FCA3E0FDA3E0FEA374
:10118700E0FFA3E0F8A3E0F9A3E0FAA3E0FB12175E
:10119700B3900291121892800A90029512189E003D
:1011A700000000900291E0F8A3E0F9A3E0FAA3E0C1
:1011B700FBAE1AAF1BE4FCFD121728900291121820
:1011C70092900291E0FCA3E0FDA3E0FEA3E0FF788C
:1011D7000A12186C900291121892E47FFF7E03FDA9
:1011E700FC900289E0F8A3E0F9A3E0FAA3E0FBC3CF
:1011F70012185B501C900289E0F8C374FF9BFF74C0
:10120700039AFEE499FDE498FC90029512189280E7
:101217000A90029512189E00000000900295E0FCCB
:10122700A3E0FDA3E0FEA3E0FF780A12187F900277
:1012370095121892C3E51994FFE5189403502F905F
:101247000295E0FCA3E0FDA3E0FEA3E0FFC006C01B
:1012570007C374FF9519FF74039518AB07FAE4F9F0
:10126700F8D007D0061217B3900295121892900281
:1012770095E0F8A3E0F9A3E0FAA3E0FBAE1CAF1DED
:10128700E4FCFD121728900295121892900295E03F
:10129700FCA3E0FDA3E0FEA3E0FF780A12186C9020
:1012A7000295121892900291E0FCA3E0FDA3E0FEE4
:1012B700A3E0FFA3E0F8A3E0F9A3E0FAA3E0FB8033
:1012C70059900289E0F8A3E0F9A3E0FAA3E0FBC391
:1012D70074FF9BFB74039AFAE499F9E498F8AE1249
:1012E700AF13E4FCFD121728780A12186CC004C06B
:1012F70005C006C007AE1AAF1BE4FCFD900289E0EB
:10130700F8A3E0F9A3E0FAA3E0FB121728780A1282
:10131700186CD003D002D001D000EF2BFFEE3AFEBD
:10132700ED39FDEC38FC900291121892900326E0FB
:10133700FCA3E0FDA3E0FEA3E0FF90028DE0F8A38D
:10134700E0F9A3E0FAA3E0FBD312185B4035900263
:101357008DE0FCA3E0FDA3E0FEA3E0FF90032612CF
:10136700189290028DE0FCA3E0FDA3E0FEA3E02429
:10137700FCFFEE34FFFEED34FFFDEC34FFFC900381
:101387002E805290032EE0FCA3E0FDA3E0FEA3E035
:10139700FF90028DE0F8A3E0F9A3E0FAA3E0FBC316
:1013A70012185B503390028DE0FCA3E0FDA3E0FE32
:1013B700A3E0FF90032E12189290028DE0FCA3E0A9
:1013C700FDA3E0FEA3E02404FFE43EFEE43DFDE4CC
:1013D7003CFC900326121892900336E0FCA3E0FD34
:1013E700A3E0FEA3E0FF900291E0F8A3E0F9A3E0F9
:1013F700FAA3E0FBD312185B4035900291E0FCA3FF
:10140700E0FDA3E0FEA3E0FF9003361218929002DE
:1014170091E0FCA3E0FDA3E0FEA3E024FCFFEE3493
:10142700FFFEED34FFFDEC34FFFC90033E8052904D
:10143700033EE0FCA3E0FDA3E0FEA3E0FF900291E2
:10144700E0F8A3E0F9A3E0FAA3E0FBC312185B50AE
:1014570033900291E0FCA3E0FDA3E0FEA3E0FF9040
:10146700033E121892900291E0FCA3E0FDA3E0FE78
:10147700A3E02404FFE43EFEE43DFDE43CFC9003CE
:101487003612189290032EE0FCA3E0FDA3E0FEA322
:10149700E0FF90028D12189290033EE0FCA3E0FD5E
:1014A700A3E0FEA3E0FF900291121892E47FFF7E73
:1014B70003FDFC90028DE0F8A3E0F9A3E0FAA3E0B6
:1014C700FBD312185B400A90028D12189E0000038E
:1014D700FFE47FFF7E03FDFC900291E0F8A3E0F9B3
:1014E700A3E0FAA3E0FBD312185B400A9002911223
:1014F700189E000003FFC28490028DE0FCA3E0FD6C
:10150700A3E0FEA3E0FF780212186C900349EEF007
:10151700A3EFF090028DA3A3A3E05403FFE4FEFD25
:10152700FC780612187FC004C005C006C007A3E0F8
:10153700FCA3E0FDA3E0FEA3E0FF780612186CD041
:1015470003D002D001D000EF4BFFEE4AFE90034BD1
:10155700EEF0A3EFF0900291A3A3A3E0543FFFE4C2
:10156700FEFDFC780212187F90034DEEF0A3EFF01A
:02157700C204AC
:01157900224F
:031A1500022F6C31
:102F6C00C0E0C083C082C0D075D000C004C005C012
:102F7C0006C007C2FF90035FE004F0C36480948333
:102F8C005007E0FF3395E0801D90035FE0FFC364C2
:102F9C008094855029A3E0FD3395E0FCEF3395E058
:102FAC00FEEF2DFFEE3CFEEF25E0FFEE33FE744905
:102FBC002FF58274033EF583A3E0F5A380139003F1
:102FCC0060E02402F0E0D3648094854002E4F0D207
:102FDC0084D007D006D005D004D0D0D082D083D0F6
:022FEC00E032D1
:031A2D000235106F
:10351000C0E0C083C082C0D075D000C00753917F87
:0E352000122FEED007D0D0D082D083D0E03270
:031A21000227E2B7
:1027E200C0E0C0F0C083C082C0D075D000C000C0BD
:0B27F20002C003C004C005C006C00701
:1027FD00C2EDAFBEEFFEADBDEDFBAA0690035DE0F1
:10280D007004A3E064027075E5BBB403047F01801E
:10281D00027F00E5BBB40D047E0180027E00EE4F09
:10282D006045D3EB94C8EA648094834018AFBBEF46
:10283D0025E024C6F582E43402F5837403F0A37415
:10284D00C8F0022909C3EB9468EA64809480AFBB99
:10285D00EF501725E024C6F582E43402F583E4F049
:10286D00A37468F0022909AFBBEF25E024C6F582F9
:10287D00E43402F583EAF0A3EBF0022909AFBBEFD4
:10288D0025E024C6F582E43402F583EAF0A3EBF0EB
:10289D0090035DE475F0011216FCFEC3E5F0940A99
:1028AD00EE64809480500990035DA3E0F5BB803603
:1028BD00900346E475F0011216FCFED3E5F0941377
:1028CD00EE64809480400B900346E4F0A3740AF00C
:1028DD00D20390035DE4F0A37402F0D2049003469A
:1028ED00A3E0540FF5BB900346E0FCA3E0FDAF035E
:0C28FD00AE021216EAAA06AB0775E8D07E
:10290900D007D006D005D004D003D002D000D0D053
:09291900D082D083D0F0D0E0326E
:10319C00420205000042020A000042020C0000C17B
:0531AC000AC10BC1097E
:0A368100C20BC20AE490024EF022D0
:1033E000E4900205F0A3F090020AF0A3F090020E20
:1033F000F090020CF0A3F0900208F0A37440F0E407
:05340000900207F0221C
:061A0C001236810233E0F6
:0D363A0075C19043E6019002037401F02277
:10360C0043C140E5C120E5FB121A0CE4900203F023
:01361C00228B
:0A368B0053C1BF9002037401F02246
:0D364700AE0712363A900204EEF0021A0CA3
:10340500E49002B7F0A3F0300B02FF22200AFDD2B0
:103415000B90024FE4F0A37410F0900252EFF0E429
:04342500A3F07F0190
:013429002280
:10333100300B0A90024FE07002A3E070037F00227D
:10334100900250E024FFF090024FE034FFF0900231
:1033510053E0FE04F074542EF582E43402F583EF59
:04336100F07F0122D6
:0B367600300B07C20BD20A123695225F
:0A369500E5C120E5FBC2C4D2C52246
:103069009002B1EBF0A3EAF0A3E9F0900203E0705B
:1030790002FF229002B4E0FE6005D3941040037F62
:083089000022123405EF604E35
:10309100E49002B6F09002B4E0FF9002B6E0FEC305
:1030A1009F50249002B1E0FBA3E0FAA3E0F98E82E5
:1030B100758300121689FF123331EF7002FF2290DF
:1030C10002B6E004F080CEE490024EF01236769023
:0E30D10002B5E07003200AFD90024EE0FF22DF
:0330DF007FFF224E
:0E2B8400900280EBF0A3EAF0A3E9F0A3EDF0DD
:102B9200E4FFD3900206E09400900205E064809482
:102BA2008050012253E6FE90020CE0FEA3E0240EC8
:102BB200F58274023EF583E0FF90020CE475F001A9
:102BC2001216FCFCE5F064404C700690020CF0A377
:102BD200F0900209E004F07006900208E004F0E4CC
:102BE200FE900283E0FDEEC39D5054EEC39F504F12
:102BF20090020CE0FCA3E0240EF58274023CF58303
:102C0200E0FD900280E0FBA3E0FAA3E0F98E82757A
:102C12008300ED1216C890020CE475F0011216FC46
:102C2200FCE5F064404C700690020CF0A3F09002B8
:102C320009E004F07006900208E004F00E80A2EEB3
:102C4200C39F502990020CE475F0011216FCFCE5BA
:102C5200F064404C700690020CF0A3F0900209E080
:102C620004F07006900208E004F00E80D290020692
:102C7200E024FFF0900205E034FFF043E601900209
:0C2C820083E0FEEFC39E50028002AF060C
:012C8E002223
:1035B200D3900206E09400900205E064809480407B
:0835C200047F0180027F00225A
:031A180002223B6C
:10223B00C0E0C0F0C083C082C0D075D000C000C069
:03224B0006C007C3
:10224E00C20DE5C054FE1218CF232A08232A0A22F3
:10225E00F10C22F10E23A31023A31222F722230244
:10226E002823022A22F72C22F72E22E4C0229DC216
:10227E002288E02288E2000023AEC209900252E0DA
:10228E00F5C2C2C5C2C490025174FFF00223B090D1
:10229E000251E0FFB4FF12900253E0F5C2C2C5C274
:1022AE00C4900251E4F00223B0900253E0FEEFC35B
:1022BE009E5017900251E0FF04F074542FF582E403
:1022CE003402F583E0F5C20223B0D2C490024EE48C
:1022DE00F0C20A0223B090024E74FDF0D2C5C2C401
:1022EE000223B090025174FFF0D209C2C4C2C1D20F
:1022FE00C50223B0E5C26007900204E0B5C20E909D
:10230E000202E4F0C2C5C2C4D2C10223B0C2C4C22A
:10231E00C13009030223A8C2C50223B0900202E015
:10232E007020E5C2F0E0FFC3900209E09F7480F8D0
:10233E00900208E064809850031233E0900202E0AD
:10234E0004F0900209E024FFF0900208E034FFF060
:10235E0090020AE0FEA3E0240EF58274023EF5839D
:10236E00E5C2F090020AE475F0011216FCFEE5F0EB
:10237E0064404E700690020AF0A3F0900202E01440
:10238E00F0700E900206E004F07006900205E00474
:10239E00F0D2C1800DC2C4300908C209D2C5800274
:1023AE00D20D300D1053C17F43C180C2C5C2C4C20D
:0723BE00C1C20DC20AC2C03A
:1023C500D007D006D000D0D0D082D083D0F0D0E0D6
:0123D50032D5
:051A1B00E5C15420FFAD
:011A200022A3
:0736AF0043C14053E6FE2277
:1025480090028EE0FFA3E0FCA3E0FDA3E0FBA3E084
:10255800FAA3E0F990029DE527F0E528A3F09002A0
:0625680096E090029FF0D6
:10256E00900297EFF0A3ECF0A3EDF0A3EBF0A3EA4B
:04257E00F0A3E9F0ED
:102582009002A07403F0A374E8F0E5C120E5FBD249
:10259200C1C2C4D2C5E4FF90037AF030C0FDE5C0E9
:1025A20054FE2440700302264524FE602424E26087
:1025B2000924FE600524E202264DC2C5EF60030233
:1025C2002653900297E025E044A0F5C27F0302263D
:1025D20053EFB4030A900298E0F5C27F058072EFD0
:1025E200B4050B900298A3E0F5C27F068063EF6406
:1025F20006703E90029FE090029A700FE0FBA3E407
:1026020075F001121712A9F0FA8008E0FBA3E0FAB4
:10261200A3E0F9121670F5C290029EE024FFF0903A
:10262200029DE034FFF0E07002A3E070247F078097
:1026320020EFB40706D2C47F09801690037A74058E
:10264200F0800E90037A7402F0800690037A74018F
:10265200F0EFB40904C2C0803690037AE0FE64064B
:102662006012EEB402169002A074FFF5F01216FC8E
:1026720045F06008D2C5E490037AF0FF90037AE057
:102682006008C2C5D2C4C2C08005C2C002259DE591
:04269200C120E5FB83
:012696002221
:1026970090028FEFF0A3ECF0A3EDF0A3EBF0A3EA29
:0426A700F0A3E9F0C3
:1026AB009002977403F0A374E8F0E5C120E5FBD228
:1026BB00C1C2C4D2C5E4FF90037AF030C0FDE5C0BF
:1026CB0054FE24C8700302278824AE607A24CA7093
:1026DB000302279024FE603824E2600924FE600583
:1026EB0024E2022798C2C5EF700F90028FE025E01D
:1026FB0044A0F5C27F0302279EEF6401600302270B
:10270B009E90028FE025E044A1F5C27F0402279E34
:10271B00EFB4030A900290E0F5C27F058075EFB429
:10272B00050B900290A3E0F5C27F068066EFB4061E
:10273B0006D2C57F01805CEFB404047F0280549005
:10274B00037A7405F0804C900292E0FBA3E475F0E1
:10275B0001121712A9F0FAE5C21216B6900296E012
:10276B0024FFF0900295E034FFF0E07002A3E070DC
:10277B00087F09C2C1D2C4801A7F02801690037AE7
:10278B007406F0800E90037A7402F0800690037A40
:10279B007401F0EFB40904C2C0803690037AE0FEF6
:1027AB0064066012EEB4021690029774FFF5F012F5
:1027BB0016FC45F06008D2C5E490037AF0FF900355
:1027CB007AE06008C2C5D2C4C2C08005C2C002266E
:0627DB00C6E5C120E5FB8C
:0127E10022D5
:102C8F0090028EEFF0900291EBF0A3EAF0A3E9F03F
:082C9F0090028FECF0A3EDF0B0
:102CA700752900543FF52A543F605CC37440952A48
:102CB700FFE49529FE900294E0FCA3E0FDC39FEC9E
:102CC7009E50068C278D2880048E278F2812254832
:102CD70090037AE060037F0222900290E02528F0BB
:102CE70090028FE03527F0900296E0700B900292E9
:102CF700E5278528F01216FCC3900295E09528F089
:102D0700900294E09527F0900294E0F527A3E0F570
:102D170028D3E5289400E52794004070E5289440DF
:102D2700E5279400501312254890037AE060037F4B
:102D37000222E4F527F52880D890028EE0FFA3E071
:102D4700FCA3E0FDA3E0FBA3E0FAA3E0F990029D5A
:102D5700E4F0744012256490037AE060037F022256
:102D670074C02528F52874FF3527F527900290E0D1
:102D77002440F090028FE03400F0900296E07091CA
:0E2D870090029275F0401216FC022D187F008B
:012D9500221B
:1035CA00900295E4F0A304F012269790037AE06043
:0735DA00037F01227F0022A4
:10354C00900379EBF07B017A037979900294E4F0A3
:0A355C00A304F0E4A3F0122C8F2268
:10344C00C00790028DE0FFA3E0900295CFF0A3EFB0
:10345C00F0D00712269790037AE060037F01227F59
:02346C0000223C
:10356600C00790028CE0FFA3E0900294CFF0A3EF97
:0A357600F0E4A3F0D007122C8F221E
:0E32A8009002AAEBF0A3EAF0A3E9F0A3EDF088
:1032B600E49002AFF09002AAE0FBA3E0FAA3E0F9E3
:1032C600A3E09002B4F09002AEE09002B5F0E4FF05
:1032D600123069EFB4FF0D9002AFE0FE04F0EEC3CA
:0632E600940340D17E00BC
:0132EC0022BF
:0B33650090027DEBF0A3EAF0A3E9F07A
:103370007E007F007D101218F590027DE0FBA3E037
:10338000FAA3E0F97D10122B84EF7002FF227F0177
:01339000221A
:1031B60090027D7422F0A3EFF0A37413F012167040
:1031C600900280F0900001121689900281F0900022
:1031D60002121689900282F090000312168990025C
:1031E60083F0900004121689900284F09000051274
:1031F6001689900285F0900006121689900286F0D4
:103206007B017A02797DE49002AEF07D0A0232A853
:10346E009002A67422F0A3EFF0A37403F0A374FFEE
:10347E00F07B017A0279A6E49002AEF07D0402326E
:01348E00A895
:10348F0090027D7422F0A3EFF0A3741CF0A374FFDD
:10349F00F07B017A02797DE49002AEF07D04023276
:0134AF00A874
:1034F100E490027DF0A3EFF0A3740AF0A3EFF07B58
:0F350100017A02797DE49002AEF07D040232A8D7
:1034B000A2AFE433FCC2AF758F0175B7A575B7F144
:1034C0008F828E83EDF0E4F58FAF04EF24FF92AF8F
:0134D00022D9
:1034D100A2AFE433FDC2AF758F0375B7A575B7F120
:0F34E1008F828E83E4F0F58FAF05EF24FF92AF5B
:0134F00022B9
:10321600900294EEF0A3EFF0A3ECF0A3EDF0EB4AEE
:103226006039900294E0FEA3E0FFA3E0FCA3E0F582
:10323600828C83E0FD1234B0EB1B70011A9002976A
:10324600E004F07006900296E004F0900295E00427
:0C325600F070CB900294E004F080C322E2
:0836A700E4900000F0A3F02202
:1033BA00900000E0FEA3E0FF1234D1900000E0FE8E
:1033CA00A3E0FF7C007D027B007A02123216E490B1
:0633DA000000F0A3F02248
:0A2EE000A90590028EEEF0A3EFF0BA
:102EEA00EE54FEFE900000E0FCA3E0FD7002EE6CE2
:102EFA006057ED4C60031233BA90028EE0FEEE5436
:102F0A00FEFE7F00900000F0A3EFF0900290EEF03A
:102F1A00A3EFF0A37400F0A37402F07E0290029073
:102F2A00E475F00112171285F082F583E493FD909F
:102F3A000292E475F00112171285F082F583EDF022
:102F4A00EF1F70011EEF4E70D490028EE0FCA3E0DA
:102F5A00FDEC5401FC74022DF58274003CF583E902
:012F6A00F076
:012F6B002243
:10326200900287EEF0A3EFF0A3EBF0A3EAF0A3E95C
:10327200F090028C74FFF5F012171245F060269060
:103282000287E475F001121712AFF0FE900289E096
:10329200FBA3E475F001121712A9F0FA121670FDE1
:0632A200122EE080CC2298
:061FE5009002A612189202
:101FEB009002AEE0FCA3E0FDA3E0FEA3E0FBAA069B
:101FFB00A905A8049002AAE0FCA3E0FDA3E0FEA3C0
:10200B00E0C39BFFEE9AFEED99FDEC98FC9002B6B7
:10201B001218929002BA12189E000000009002B69D
:10202B00E0FCEC3340030220EB9002AEE0FCA3E0BB
:10203B00FDA3E0FEA3E0FF9002C2121892E47F0121
:10204B00FEFDFC9002C2E0F8A3E0F9A3E0FAA3E0E6
:10205B00FBC3121845500A9002C212189E000000D2
:10206B00019002A6E0FCA3E0FDA3E0FEA3E0FF903D
:10207B0002B2E0F8A3E0F9A3E0FAA3E0FB12172801
:10208B00C004C005C006C0079002C2E0FCA3E0FD7F
:10209B00A3E0FEA3E0FBAA06A905A804D007D0067F
:1020AB00D005D0041217B39002BE1218929002BE44
:1020BB00E0FCA3E0FDA3E0FEA3E0FF9002AAE0F8A2
:1020CB00A3E0F9A3E0FAA3E0FB1217289002B2E019
:1020DB00F8A3E0F9A3E0FAA3E0FB1217B302222660
:1020EB00E4FFFEFDFC9002B6E0F8A3E0F9A3E0FAF2
:1020FB00A3E0FBD3121845500302222C9002A6E05A
:10210B00F8A3E0F9A3E0FAA3E0FB9002B2E0FCA392
:10211B00E0FDA3E0FEA3E09BFFEE9AFEED99FDEC44
:10212B0098FC9002B2E0F8A3E0F9A3E0FAA3E0FB7D
:10213B001217289002BE1218929002AEE0FCA3E098
:10214B00FDA3E0FEA3E0FBAA06A905A804A3E0FCFF
:10215B00A3E0FDA3E0FEA3E0C39BFFEE9AFEED9987
:10216B00FDEC98FC9002C2121892E47F01FEFDFC7C
:10217B009002C2E0F8A3E0F9A3E0FAA3E0FBC312DC
:10218B001845500A9002C212189E000000019002DE
:10219B00BEE0FCA3E0FDA3E0FEA3E0FFA3E0F8A3F9
:1021AB00E0F9A3E0FAA3E0FB1232ED9002BE1218A5
:1021BB00929002AAE0F8A3E0F9A3E0FAA3E0FB9067
:1021CB0002B2E0FCA3E0FDA3E0FEA3E0C39BFBEEA9
:1021DB009AFAED99F9EC98F89002BEE0FCA3E0FDB9
:1021EB00A3E0FEA3E0FF1217289002B2E0F8A3E0F1
:1021FB00F9A3E0FAA3E0FB1217B3AB07AA06A905F4
:10220B00A8049002B2E0FCA3E0FDA3E0FEA3E0C3B0
:10221B009BFFEE9AFEED99FDEC98FC9002BA12181A
:0F222B00929002BAE0FCA3E0FDA3E0FEA3E0FF67
:01223A002281
:102922009002A6EFF025E024FCF582E43402F58360
:10293200E0FEA3E0FFE4FCFD9002A7E0F8A3E0F9CB
:10294200A3E0FAA3E0FBD312185B40339002A7A3E3
:10295200A3E0FEA3E0FF9002A6E0FD25E024FCF543
:1029620082E43402F583EEF0A3EFF0EF24FCFFEEF5
:1029720034FFFEED25E02410F582E43403806A90F2
:1029820002A6E025E02410F582E43403F583E0FE9C
:10299200A3E0FFE4FCFD9002A7E0F8A3E0F9A3E0C6
:1029A200FAA3E0FBC312185B50469002A7A3A3E070
:1029B200FEA3E0FF9002A6E0FD25E02410F582E4EC
:1029C2003403F583EEF0A3EFF0ED25E02410F58259
:1029D200E43403F583E0FEA3E02404FFE43EFEEDCD
:1029E20025E024FCF582E43402F583EEF0A3EFF057
:1029F2009002A6E025E02410F582E43403F583E09A
:102A0200FEA3E0FFE4FCFD9002A71218929002AB35
:102A1200E0FCA3E0FDA3E0FEA3E0FF9002A7E0F844
:102A2200A3E0F9A3E0FAA3E0FBD312185B401490F1
:102A320002ABE0FCA3E0FDA3E0FEA3E0FF9002A74F
:102A42001218929002A7E0FCA3E0FDA3E0FEA3E02F
:022A5200FF2261
:052A540090029DEFF06F
:102A5900C007ED25E024C6F582E43402F583E0FEE3
:102A6900A3E0FFE4FCFD9002A71218929002AB12BA
:102A7900189E000003FFD00712292290029E121807
:102A89009290029DE025E024E8F582E43402F58382
:102A9900E0FEA3E0FFE4FCFD90029EE0F8A3E0F96C
:102AA900A3E0FAA3E0FBC312185B7003022B839027
:102AB900029DE025E0240AF8E6FE08E6FFE4FCFDB5
:102AC900C004C005C006C007A3E0FCA3E0FDA3E065
:102AD900FEA3E0FF9002AA12189290029DE025E061
:102AE90024E8F582E43402F583E0FEA3E0FFE4FC88
:102AF900FD9002AE1218929002B212189E000003C5
:102B0900FFD007D006D005D004121FE59002A2120B
:102B1900189290029DE025E0240AF8E6FE08E6FFF7
:102B2900E4FCFD9002A2E0F8A3E0F9A3E0FAA3E037
:102B3900FBC312185B60259002A2A3A3E0FEA3E0E9
:102B4900FF90029DE025E0240AF8A60608A6079052
:102B590002E6E07002A3E0700312352E90029EA3F4
:102B6900A3E0FEA3E0FF90029DE025E024E8F582C2
:0A2B7900E43402F583EEF0A3EFF060
:012B8300222F
:0431B1004103620074
:0636BD00E4900362F0221C
:0736B6009003627401F02291
:1030E20090027D7404F0E4A3F0A3F01236A77E39B7
:1030F2007F007B017A02797D90028CE4F0A304F0D8
:10310200123262E490027EF090027EE0FFC3941ECF
:10311200502A75F016EFA42401F582E5F03439AF98
:1031220082FE7B007A00790890028CE4F0A3741688
:10313200F012326290027EE004F080CC7E3B7F95FA
:103142007B017A02797F90028CE4F0A304F01232C0
:04315200620233BA28
:10352E00200C1A300713308712900362E0700C9053
:0E353E000348E0FF12346E8002D287D20C22C6
:10358000903B95E493F46009903900E493640460FF
:0A359000031230E2E4900361F02220
:10339100900361E0FFC3941E501EEF75F016A42444
:1033A10001F9743935F0FA7BFF78087C007D007EE5
:0933B100007F1612164AC20C221C
:1019D700900361E0C3941E502B1236A7900361E079
:1019E70075F016A42401F582E5F03439AF82FE7B49
:1019F700007A00790890028CE4F0A37416F0123292
:051A0700621233BA2257
:0636C3001219D7C20C220F
:052D960090027EEDF04B
:102D9B00900280E004F0900283EFF0A3EBF090023E
:102DAB007EE0FF900283E0FED39F4003022E497525
:102DBB00F016EEA42401F582E5F03439AF829002CF
:102DCB0085F0A3EFF0900284E075F016A42401F5D2
:102DDB0082E5F03439AF82900287F0A3EFF0E490F4
:102DEB000281F0A3F0900287E475F001121712AF85
:102DFB00F0FE900285E0FCA3E0F5828C83E493FD6A
:102E0B00122EE0900286E004F07006900285E0043A
:102E1B00F0900282E004F07006900281E004F0C3AF
:102E2B00900282E09416900281E0940040B7123336
:0E2E3B00BA900283E004F0A3E004F0022DA997
:012E49002266
:0523D60090027DEDF016
:1023DB00900282EFF0A3EBF090027DE0FF9002827F
:1023EB00E0D39F4003022547A3E075F016A4240118
:1023FB00F582E5F03439AF8290027EF0A3EFF0E482
:10240B00900284F0A3F0900284E0FEA3E0FFC3945B
:10241B0016EE9400503890027EE0FCA3E0F5828C1F
:10242B0083E493FD74632FF582E43403F583EDF0BD
:10243B0090027FE004F0700690027EE004F09002C0
:10244B0085E004F070C0900284E004F080B8900244
:10245B0082E075F016A42401F582E5F03439AF82E1
:10246B00900280F0A3EFF0900283E075F016A424A5
:10247B0001F582E5F03439AF8290027EF0A3EFF0E4
:10248B00E4900284F0A3F090027EE475F001121741
:10249B0012AFF0FE900280E0FCA3E0F5828C83E4A7
:1024AB0093FD122EE0900281E004F0700690028002
:1024BB00E004F0900285E004F07006900284E004E2
:1024CB00F0C3900285E09416900284E0940040B72C
:1024DB00900282E075F016A42401F582E5F0343900
:1024EB00AF82900280F0A3EFF0E4900284F0A3F0AF
:1024FB00900284E0FCA3E0FDC39416EC9400502CF6
:10250B00900280E475F001121712AFF0FE74632D88
:10251B00F582E43403F583E0FD122EE0900285E0B2
:10252B0004F070CC900284E004F080C41233BA90B3
:0C253B000282E004F0A3E004F00223E3BD
:012547002271
:0B19210090027DEFF0A3EDF0A3EBF0CF
:10192C00A2AFE433A3F0C2AF1236AF90027EE0FE5A
:10193C0090027DE0FDEDFF900285EEF0A3EFF0E468
:10194C00900281F090027FE0FF900285E0FCA3E022
:10195C00FD7B017A03796390028DE4F0A37416F099
:10196C0012344C900286E02416F0900285E034008C
:10197C00F0900281E075F016A42401F9743935F069
:10198C00FAA374FFF0A3EAF0A3E9F01236A79002D1
:10199C0082A3E0FAA3E0AE02FF7B017A03796390A5
:1019AC00028CE4F0A37416F01232621233BA900275
:1019BC0081E004F0E0C3941E408A900348E0FF12DB
:0A19CC003647900280E024FF92AF3E
:0119D60022EE
:0B2E4A0090027DEFF0A3EDF0A3EBF091
:102E5500A2AFE433A3F0C2AF1236AF90027EE0FE1C
:102E650090027DE0FDEDFF900282EEF0A3EFF0E42D
:102E7500900281F0900281E0FFC3941E504C75F0E2
:102E850016EFA42401F582E5F03439AF82FE9002F5
:102E950084F0FAA3EFF0FB90027FE0FF900282E05E
:102EA500FCA3E0FDA9037BFF90028CE4F0A374165C
:102EB500F0123566900283E02416F0900282E03429
:102EC50000F0900281E004F080AA900348E0FF1230
:0A2ED5003647900280E024FF92AF20
:012EDF0022D0
:03000000020800F3
:03000300021A03DB
:03000B00021A06D0
:03001300021A09C5
:03001B00021A0CBA
:03002300021A0FAF
:03002B00021A12A4
:03003300021A1599
:03003B00021A188E
:03004300021A1B83
:03004B00021A1E78
:03005300021A216D
:03005B00021A2462
:03006300021A2757
:03006B00021A2A4C
:03007300021A2D41
:10080000E4F5D9E5EF7480F5FF7402F5EF787FE445
:10081000F6D8FD9000007F007E04E4F0A3DFFCDE4C
:07082000FA75812A0208624B
:10082700021D53E493A3F8E493A34003F68001F277
:1008370008DFF48029E493A3F85407240CC8C333D2
:10084700C4540F4420C8834004F456800146F6DFA1
:10085700E4800B0102040810204080903156E47EAA
:10086700019360BCA3FF543F30E509541FFEE49396
:10087700A360010ECF54C025E060A840B8E493A35D
:10088700FAE493A3F8E493A3C8C582C8CAC583CA88
:10089700F0A3C8C582C8CAC583CADFE9DEE780BE40
:0131B5000019
:10157A00E709F608DFFA8046E709F208DFFA803E53
:10158A0088828C83E709F0A3DFFA8032E309F60840
:10159A00DFFA8078E309F208DFFA807088828C83A8
:1015AA00E309F0A3DFFA806489828A83E0A3F6085C
:1015BA00DFFA805889828A83E0A3F208DFFA804C36
:1015CA0080D280FA80C680D4806980F2803380100D
:1015DA0080A680EA809A80A880DA80E280CA803376
:1015EA0089828A83ECFAE493A3C8C582C8CCC583EE
:1015FA00CCF0A3C8C582C8CCC583CCDFE9DEE780BE
:10160A000D89828A83E493A3F608DFF9ECFAA9F03C
:10161A00EDFB2289828A83ECFAE0A3C8C582C8CC92
:10162A00C583CCF0A3C8C582C8CCC583CCDFEADEAB
:10163A00E880DB89828A83E493A3F208DFF980CC0D
:10164A0088F0EF60010E4E60C388F0ED2402B40406
:10165A000050B9F582EB2402B4040050AF232345AD
:06166A0082239015CA73F3
:10167000BB010689828A83E0225002E722BBFE0278
:09168000E32289828A83E49322AB
:10168900BB010CE58229F582E5833AF583E0225016
:1016990006E92582F8E622BBFE06E92582F8E22260
:0D16A900E58229F582E5833AF583E493227A
:1016B600BB010689828A83F0225002F722BBFE0113
:0216C600F3220D
:1016C800F8BB010DE58229F582E5833AF583E8F058
:1016D800225006E92582C8F622BBFE05E92582C804
:0216E800F222EC
:1016EA00EF8DF0A4A8F0CF8CF0A428CE8DF0A42E14
:0216FA00FE22CE
:1016FC00C5F0F8A3E028F0C5F0F8E5821582700279
:06170C001583E038F02215
:10171200A3F8E0C5F025F0F0E5821582700215838A
:06172200E0C838F0E822E7
:10172800E88FF0A4CC8BF0A42CFCE98EF0A42CFC60
:101738008AF0EDA42CFCEA8EF0A4CDA8F08BF0A4DE
:101748002DCC3825F0FDE98FF0A42CCD35F0FCEB3D
:101758008EF0A4FEA9F0EB8FF0A4CFC5F02ECD3902
:0F176800FEE43CFCEAA42DCE35F0FDE43CFC226F
:1017770075F008758200EF2FFFEE33FECD33CDCC29
:1017870033CCC58233C5829BED9AEC99E5829840AC
:101797000CF582EE9BFEED9AFDEC99FC0FD5F0D689
:1017A700E4CEFBE4CDFAE4CCF9A88222B800C1B9B3
:1017B7000059BA002DEC8BF084CFCECDFCE5F0CBF1
:1017C700F97818EF2FFFEE33FEED33FDEC33FCEB2A
:1017D70033FB10D703994004EB99FB0FD8E5E4F9E5
:1017E700FA227818EF2FFFEE33FEED33FDEC33FCD2
:1017F700C933C910D7059BE99A4007EC9BFCE99AC6
:10180700F90FD8E0E4C9FAE4CCFB2275F010EF2F0A
:10181700FFEE33FEED33FDCC33CCC833C810D7070A
:101827009BEC9AE899400AED9BFDEC9AFCE899F845
:0E1837000FD5F0DAE4CDFBE4CCFAE4C8F922D8
:1032ED00C2D5E830E70FB2D5E4C39BFBE49AFAE40C
:1032FD0099F9E498F8EC30E717B2D5123323121789
:10330D00B3E4C39BFBE49AFAE499F9E498F88003DB
:10331D001217B330D50DE4C39FFFE49EFEE49DFD6F
:04332D00E49CFC22FE
:10184500EB9FF5F0EA9E42F0E99D42F0EC6480C81A
:0618550064809845F022BA
:10185B00EB9FF5F0EA9E42F0E99D42F0E89C45F0E3
:01186B00225A
:10186C00E8600FECC313FCED13FDEE13FEEF13FF5A
:03187C00D8F1227E
:10187F00E8600FEFC333FFEE33FEED33FDEC33FCC7
:03188F00D8F1226B
:0C189200ECF0A3EDF0A3EEF0A3EFF022C9
:10189E00A8828583F0D083D0821218B51218B512A3
:1018AE0018B51218B5E473E493A3C583C5F0C583C8
:1018BE00C8C582C8F0A3C583C5F0C583C8C582C894
:0118CE0022F7
:1018CF00D083D082F8E4937012740193700DA3A3A8
:1018DF0093F8740193F5828883E4737402936860BC
:0618EF00EFA3A3A380DFBC
:1018F500EF4E6012EF60010EEDBB010B89828A830A
:10190500F0A3DFFCDEFA2289F05007F709DFFCA916
:0C191500F022BBFEFCF309DFFCA9F0226D
:00000001FF
